:100000000C9447040C947F040C947F040C947F049C
:100010000C947F040C947F040C947F040C947F0454
:100020000C947F040C947F040C9474220C94302262
:100030000C9471230C947F040C947F040C947F0423
:100040000C947F040C947F040C947F040C947F0424
:100050000C947F040C944D230C947F040C947F0427
:100060000C947F040C947F040C947F040C947F0404
:100070000C947F040C947F040C947F040C947F04F4
:100080000C947F040C947F040C947F040C947F04E4
:100090000C947F040C947F040C947F040C947F04D4
:1000A0000C947F040C947F040C947F0405010902D6
:1000B000A10185020901A1000509190129081500FE
:1000C0002501950875018102050109300931158165
:1000D000257F95027508810609381581257F9501D0
:1000E00075088106050C0A38021581257F95017572
:1000F000088106C0C005010980A101850319012AF4
:10010000B700150126B700950175108100C0050CD8
:100110000901A101850419012AA002150126A002E6
:10012000950175108100C005010906A1018506052C
:100130000719E029E71500250195087501810205D9
:1001400007190029EF1500250195F07501810205B9
:10015000081901290595057501910295017503910D
:1001600001C00660FF0961A1010962150026FF00B8
:100170009520750881020963150026FF00952075FA
:10018000089102C005010906A101050719E029E748
:1001900015002501950875018102950175088101F9
:1001A0000507190029FF150026FF0095067508812F
:1001B000000508190129059505750191029501753C
:1001C000039101C0000000000000000000000000DA
:1001D000000000000000000000000000000000001F
:1001E00000000000000000007E0F00D4FFFFFFC7EA
:1001F0000000007800000000000000002A2B28000A
:1002000000000000000000000000000000000029C5
:10021000000000002C1E3420212224342627252E05
:10022000362D3738271E1F2021222324252633333D
:10023000362E37381F0405060708090A0B0C0D0E69
:100240000F101112131415161718191A1B1C1D2F35
:100250003130232D350405060708090A0B0C0D0E55
:100260000F101112131415161718191A1B1C1D2F15
:100270003130354C00047F3F1F64321464321478EF
:100280003C1E1E140A0500010101010101010101CA
:100290000202020202020202020303030303030337
:1002A0000304040404040404050505050506060604
:1002B0000606070707070708080808090909090AC1
:1002C0000A0A0B0B0B0C0C0C0D0D0D0E0E0E0F0F66
:1002D0000F101011111112121313141415151616F4
:1002E0001717181819191A1A1B1B1C1D1D1E1E1F63
:1002F0002020212222232424252626272829292AB2
:100300002B2C2D2D2E2F30313232333435363738D9
:10031000393A3B3C3D3E3F404142434445464748D5
:10032000494A4C4D4E4F50515354555658595A5BAB
:100330005D5E5F616264656668696B6C6D6F70724B
:10034000737577787A7B7D7E8082838587888A8CB7
:100350008E8F91939596989A9C9EA0A2A3A5A7A9EB
:10036000ABADAFB1B3B5B7BABCBEC0C2C4C6C9CBE2
:10037000CDCFD1D4D6D8DBDDDFE2E4E7E9EBEEF098
:10038000F3F5F8FAFDFFFFAA7F5540222325262822
:10039000292A2C2D2F3032333536383A3B3D3E401A
:1003A00042434547494A4C4E5051535557595A5C60
:1003B0005E6062646668696B6D6F71737577797B77
:1003C0007D7F81838587898A8C8E90929496989A76
:1003D0009C9E9FA1A3A5A7A8AAACAEAFB1B3B4B68B
:1003E000B8B9BBBCBEBFC1C2C3C5C6C7C9CACBCCE6
:1003F000CDCED0D1D2D2D3D4D5D6D7D7D8D9D9DAB9
:10040000DADBDBDBDCDCDCDCDCDDDDDDDDDCDCDC2D
:10041000DCDCDBDBDBDADAD9D9D8D7D7D6D5D4D355
:10042000D2D2D1D0CECDCCCBCAC9C7C6C5C3C2C12A
:10043000BFBEBCBBB9B8B6B4B3B1AFAEACAAA8A787
:10044000A5A3A19F9E9C9A98969492908E8C8A893F
:10045000878583817F7D7B79777573716F6D6B691C
:1004600068666462605E5C5A5957555351504E4CF1
:100470004A4947454342403E3D3B3A3836353332A0
:10048000302F2D2C2A292826252322E000E300E204
:10049000005100500001512C000151E600E10064C0
:1004A000001D001B00060019000500110010003996
:1004B0000004001600070009000A000B000D000EE2
:1004C000002B0014001A000800150017001C00186B
:1004D000000C0035001E001F002000210022002318
:1004E000002400250029003A003B003C003D003E6E
:1004F000003F0040004100580063006200005C566D
:100500000000004F000000000058005B005A00523D
:1005100000E500380059003700360057005E005DE6
:10052000000000310034005C0033000F0056006111
:10053000006000280030002F005F001300120055FB
:10054000005400530031002E002D002A0027002601
:10055000004E004B004D004600450044004A004359
:100560000042000100010001000100010001000142
:1005700000010001000100010001000100BD5CBF9D
:100580005CBE5C01000100BF5C01000100010001D4
:100590000001000100010001000100C25C0100C374
:1005A0005CC55CC65CC75CC85CC95C01000100013D
:1005B00000010001000100010001000100005C01D8
:1005C0000001000100010001000100010001000123
:1005D0000001000100010001000000010000000016
:1005E0000001000100010001000100010001000103
:1005F00000010001000100010000000100010001F4
:1006000000010001000100010001000100010001E2
:100610000001000100CA5C010001000100010001AD
:1006200000010001000100010001000100A900A873
:100630000001000100AA0001000100010001000109
:1006400000010001000100010001000100010001A2
:100650000001000100010001000100010001000192
:100660000001000100010001000100010001000182
:100670000001000100010001000100010001000172
:100680000001000100010001000100010001000162
:100690000001000100010001000100010001000152
:1006A0000001000100010001000100010001000142
:1006B0000000000100000000000100010001000135
:1006C0000001000100010001000100010001000122
:1006D0000000000100010001000100010001000113
:1006E0000001000100010001000100010001000102
:1006F00000010001000100010001000100010001F2
:1007000000010001000100010001000100010001E1
:1007100000010001000100010001000100010001D1
:1007200000010001000100010001000100010001C1
:1007300000010001000100010001000100010001B1
:1007400000010001000100010001000100010001A1
:100750000001000100010001000100010001000191
:100760000001000100010001000100010001000181
:100770000001000100010001000100010001000171
:100780000001000100010001000000010000000064
:100790000001000100010001000100010001000151
:1007A0000001000100010001000000010001000142
:1007B0000001000100010001000100010001000131
:1007C0000001000100010001000100010001000121
:1007D0000001000100010001000100010001000111
:1007E000000100010001000100010009025B00039B
:1007F0000100A0FA09040000010301010009211110
:1008000001000122400007058103080001090401DD
:10081000000203000000092111010001222200074B
:1008200005820320000107050303200001090402DB
:1008300000010300000009211101000122B6000798
:1008400005840320000112010002000000084D5938
:10085000964D01000102000124034D0065006C006B
:100860006F006400790039003600200053006F00EB
:100870006C006400650072006500640000000A03FB
:1008800059004D0044004B000000040309041124EA
:100890001FBECFEFDAE0DEBFCDBF04B603FE18C047
:1008A0008091270390912803A0912903B0912A03F6
:1008B0008730904BA740B04B59F410922703109209
:1008C00028031092290310922A03E0E0F8E3099527
:1008D00011E0A0E0B1E0EAE5F5E502C005900D9277
:1008E000A639B107D9F723E0A6E9B1E001C01D920E
:1008F000A732B207E1F70E9498230C94822A0C9445
:100900000000E8EDF0E080818E7F80831092E200AD
:100910001092DA001092E100A0EEB0E08C918160BC
:100920008C9380818F77808319BCA7EDB0E08C9188
:100930008E7F8C9380818F7E80831092F402089545
:100940002091E4003091E50095E6A9012091EC00AA
:10095000822F817020FF06C08091E80080FF06C0D2
:1009600080E008952091E80022FD1AC080911903CB
:10097000882389F0853089F08091EB0085FD0FC0D8
:100980002091E4003091E50042175307F9F29150AD
:10099000E1F684E0089582E0089583E0089581E01F
:1009A0000895EF92FF920F931F93CF937C018B01D9
:1009B0000E94A004C82F811117C08091E80085FD16
:1009C0000BC08091E8008E778093E8000E94A0041D
:1009D000882399F3C82F08C0F70181917F01809384
:1009E000F1000150110949F78C2FCF911F910F9100
:1009F000FF90EF90089580911B0387FF13C08091B3
:100A0000E80082FF06C08091E8008B778093E800C1
:100A100004C0809119038111F2CF089580911903C8
:100A20008823D9F38091E80080FFF8CF8091E80017
:100A30008E77ECCF982F9093E900242F762F50E0FB
:100A4000891731F07091EC002091ED005091F00089
:100A500021FD07C09F5F973071F78093E90081E027
:100A600008953091EB003E7F3093EB003091ED0024
:100A70003D7F3093ED003091EB0031603093EB001F
:100A80007093EC002093ED005093F0002091EE0065
:100A900027FDE0CF80E00895B0E0A0E0E2E5F5E0DA
:100AA0000C94E729C8EDD0E088818F7E8883E7ED3C
:100AB000F0E080818160808384E082BF81E0809368
:100AC000F40288818E7F888302EE10E0F8011082A4
:100AD0001092DA0081EEC82ED12CF60110828881A6
:100AE0008F77888388818068888388818F7D8883D9
:100AF00019BC1092190310921A0310921803109245
:100B0000170390EEE92EF12CF70180818B7F808313
:100B100088818160888342E060E080E00E941A055D
:100B2000F60180818E7F8083F801808181608083DF
:100B3000808188608083F70180818E7F80838881B7
:100B400080618883CDB7DEB7E8E00C94032AFC010E
:100B5000809121039091220386179707A0F06115D9
:100B6000710529F49091E8009E779093E80090E059
:100B70006115710551F4911108C08091E80082FF60
:100B800034C080E00895BC01F2CF8091190388231E
:100B9000C1F18530C1F18091E80083FD30C08091C2
:100BA000E80082FDEACF8091E80080FFE1CF8091EC
:100BB000F3002091F200382F6115710519F02830EB
:100BC000310558F091E02830310509F090E020918E
:100BD000E8002E772093E800CBCF81918093F1003D
:100BE000615071092F5F3F4FE7CF80911903882330
:100BF00041F0853041F08091E80083FFBECF81E075
:100C0000089582E0089583E0089508958091F602A2
:100C100008959C014FB7F8948091EB029091EC02FB
:100C2000A091ED02B091EE024FBF821B930B08958D
:100C30002FB7F8948091EB029091EC02A091ED0215
:100C4000B091EE022FBF08952091E8023091E902A1
:100C50002817390771F09093E9028093E802E09138
:100C6000E602F091E702309721F00084F185E02D53
:100C7000099508952091E4023091E502281739077B
:100C800071F09093E5028093E402E091E602F09126
:100C9000E702309721F00680F781E02D099508954D
:100CA000E091E602F091E702309729F00190F0819F
:100CB000E02D0995089580E008958F929F92AF925C
:100CC000BF92EF92FF920F931F93CF93DF938630E3
:100CD000B8F5811136C0909180009F7D909380007F
:100CE0002E98A0918600B0918700282F30E00E94B6
:100CF000B42925E030E040E050E00E947D298901E0
:100D00009A0180918600909187006CE070E00E94CB
:100D1000552960177107D8F0C80169E070E00E949A
:100D2000552970938B0060938A00DF91CF911F91BA
:100D30000F91FF90EF90BF90AF909F908F9008958C
:100D400085E090918000906290938000CACF80915E
:100D5000860090918700E0908600F0908700E091F7
:100D60008600F0918700C6E0D0E0BE010E945529C0
:100D7000060F171F211D311D4801590185E0880C00
:100D8000991CAA1CBB1C8A95D1F7C701BE010E9401
:100D900055299F0150E040E0260F371F411D511D8E
:100DA000C501B4010E947D2949015A01E0918600E4
:100DB000F0918700CA01B9010E9437299B01AC015B
:100DC000DF010E94CA299B01AC01C501B4010E9448
:100DD00037292FE096958795779567952A95D1F7CE
:100DE000009186001091870030E020E00617170779
:100DF0002807390708F095CF609186007091870029
:100E000090CF282F220F220F220F9091E30297708C
:100E1000922B9093E302987F21E009F420E09091D7
:100E2000E30220FB90F99093E3020E945D0608958F
:100E3000FA01811101C0FB0109950895089580917F
:100E4000DE02982F9E7F29F4817082608093DE02FB
:100E500008958A34E8F381708864F8CFAF92BF9226
:100E6000DF92EF92FF920F931F93CF93DF93082FA0
:100E7000162FE901E42FF0E0EA57FD4F611110C091
:100E8000E4915E2F4E2F4983E8835A83DF91CF91FF
:100E90001F910F91FF90EF90DF90BF90AF9008955A
:100EA000E62EF12C4491D42EE42FF0E026E0829F30
:100EB000C00111242FEF30E0B9010E945529802F85
:100EC00090E0880F991F55E5569FD001579FB00DB0
:100ED00011248A1B9B0B982F990F890F5901AE186B
:100EE000BF08AE9ED001AF9EB00DBE9EB00D1124C6
:100EF0005B2F189F80011124012F11275901A01A7F
:100F0000B10AAE9E8001AF9E100DBE9E100D112441
:100F10005901A81AB108AE9CC001AF9C900DBE9CAF
:100F2000900D1124892F9927281B390B2E9FC00162
:100F30002F9F900D3E9F900D1124E92F6230710577
:100F4000A1F050F46115710509F49DCF6130710570
:100F500081F0EB2F512F97CF6430710569F080F04D
:100F60006630710509F48FCFF4CFE42F4B2F592F42
:100F70008ACFE42F412F87CFEB2F542F492F83CFD8
:100F80004B2F5D2DE12F7FCF0E9418069C01909181
:100F9000990280919A02982B21F030939602209327
:100FA000950290919B0280919C02982B21F03093A6
:100FB000940220939302E091E602F091E7023097C9
:100FC00049F082E0809397020480F581E02D87E963
:100FD00092E00995089540919902803F59F48091DB
:100FE0009A0287FF0DC010929A0241110BC0109215
:100FF000910208C0813F81F480919A0218169CF3F7
:10100000442381F080919B0290919C02892B09F0EE
:101010005AC0109290020895823F49F447FFF0CFE2
:101020001092990280919A028111ECCFE0CF833F18
:1010300019F41416ACF3E4CF90919B02893F29F484
:101040001916F4F610929B02DBCF8A3F19F497FF32
:10105000D7CFF8CF90919C028B3F29F497FFD0CF48
:1010600010929C02CDCF8C3F19F41916CCF3C8CF47
:101070009CE0980F953090F4845F990B21E030E06C
:10108000B90102C0660F771F8A95E2F7CB01809500
:1010900090919802892380939802B2CF8D3F31F4CA
:1010A000809192028E7F80939202AACF8E3F21F48C
:1010B000809192028D7FF7CF8F3F09F0A1CF809171
:1010C00092028B7FF0CF08958091920280FD16C02E
:1010D00081FD16C082FD16C0809190028823A1F088
:1010E000883280F428E0829FC001112468E270E019
:1010F0000E946929862F672B39F0089582E00895B0
:1011000084E0089588E0089581E008958091920236
:1011100080FD14C081FD14C082FD16C08091910233
:10112000882381F08E3180F420E5829FC001112454
:101130006EE170E00E946929862F089584E1089588
:1011400088E2089588E0089580E50895803F31F4AD
:101150000E948608819580939A020895813F19F430
:101160000E948608F8CF823F31F40E94860881955C
:10117000809399020895833F19F40E948608F8CF5E
:10118000893F29F40E94640880939B0208958A3F56
:1011900021F40E9464088195F7CF8B3F31F40E94BF
:1011A0006408819580939C0208958C3F19F40E94F5
:1011B0006408F8CF9CE0980F953070F4845F990B29
:1011C00021E030E001C0220F8A95EAF78091980271
:1011D000822B8093980208958D3F31F48091920282
:1011E00081608093920208958E3F21F48091920253
:1011F0008260F7CF8F3FB9F7809192028460F1CF80
:1012000080E00895F894E82FE295EF70F0E031A1C6
:10121000282F2F7081E090E001C0880F2A95EAF70F
:10122000982F9095932391A392A1892B82A37894D0
:1012300008959091EF0292FF06C0282F2871283060
:10124000F9F4877F846093FF06C0282F2871283126
:10125000F1F4877E84612091F00220FF06C0382FD0
:1012600038713830D9F4877F816021FF06C0282F7C
:1012700028712831D1F4877E816194FD877E08959D
:10128000282F24712430F9F68B7F8860DCCF282F3B
:101290002471243101F78B7E8861DDCF382F3171C5
:1012A000313019F78E7F8860E0CF282F21712131EE
:1012B00021F78E7E8861E1CFCF93DF93EC018238F6
:1012C0009105B1F108F040C08133910509F49DC04A
:1012D00048F58932910509F48DC08A9709F49CC0BC
:1012E000C11521E5D20708F0C3C0C11530E5D30709
:1012F00008F01EC1C83ED10508F0A3C0C13ED1050B
:1013000088F5C83AD10508F08EC0C53AD10508F075
:1013100007C1C130D10531F1209721F1C430D10589
:1013200008F545C08533910509F45FC0C997C1F63A
:101330008091EF02837009F043C18091F00283FF36
:1013400011C0C9E2D0E00EC0833E910599F170F45E
:10135000803E910501F1823E910511F68091EF02E8
:1013600082FD21C0CE01DF91CF910895863E910587
:1013700061F1873E910571F1843E910509F0B0CF8E
:101380008091F00281FFEECF8091EF02C7EED0E0B6
:1013900084FD0DC0E7CF8091EF0280FD33C09091B6
:1013A000F00290FFDFCFC3EED0E084FFDBCFD0E0D0
:1013B000C0E0D8CF8091EF0282FDFFC09091F00293
:1013C00090FDFEC084FFCECFF2CF8091EF0283FD6F
:1013D000DDCFC8CF8091EF0283FDF5C09091F00280
:1013E00091FFF0CFC4EED0E0BDCF8091EF0285FF3A
:1013F000B9CFA7CF8091EF0285FDE8C08091F002C0
:1014000083FFB0CFC9E3D0E0ADCF8091EF0286FF7C
:10141000A9CFCAE2D0E0A6CF8091EF0286FFA2CF8B
:10142000C1E3D0E09FCFCF3BD10508F6C85AD0E04A
:10143000CC0FDD1FC25EDE4F0990D881C02DD46471
:1014400091CFC11540E2D40758F4C11581E0D80707
:1014500008F088CFC03FD10508F4A9CFD06582CF6E
:10146000C11520E4D20708F4A2CFDF70D06A7ACF8A
:10147000C11535E5D30718F5C11544E5D40708F0C3
:1014800084C0C11583E5D80708F06BC0C11522E5FB
:10149000D20708F461C0CE018370992721E030E0C3
:1014A00002C0220F331F8A95E2F7C695C69580E2E7
:1014B000C89FE0011124C22BD32BDC6853CFC11588
:1014C00039E5D307A8F4C11548E5D40708F062C090
:1014D000C11586E5D80708F06ACF8C2F0E9419093C
:1014E000C82FD0E0DC2FCC27CC27DF71D0623ACFD9
:1014F000C1152AE5D20708F452C0CE0190568115D5
:10150000904208F054CF8D2F8F710E94190990E0FE
:10151000982F882788279F719C012C2BE901E6CF03
:10152000C55AD0E0C55EDE4FC881D0E0D0641ACF86
:10153000CE018370992721E030E002C0220F331FD3
:101540008A95E2F7C695C69540E2C49FE001112452
:10155000C22BD32BDD6806CFDC2FCC27C16FD06A1E
:1015600001CFCE018370992721E030E002C0220F25
:10157000331F8A95E2F7C695C69540E2C49FE00105
:101580001124C22BD32BDA68EDCEDC2FCC27C46F0D
:10159000D06AE8CEDC2FCC27C06FD06AE3CE8C2F88
:1015A0008F700E94190934E0D695C7953A95E1F7F6
:1015B000CF709C2FEC01D069D5CEC2EED0E0D2CE58
:1015C000C0EED0E0CFCEC6EED0E0CCCEC5E3D0E0CA
:1015D000C9CE80913E02811110923E0208958095FD
:1015E00090913D02982390933D02089590911A01A5
:1015F0009923D1F09091EF0297FF16C0E82FE6955E
:10160000E695E695EE31E0F4F0E0E856FE4F282F3F
:10161000277081E090E001C0880F2A95EAF7809555
:101620009281892382830895EAE9F1E091918913F7
:1016300003C0DF0111971C9291E0E03AF907B1F77E
:10164000089590911A019923C1F09091EF0297FFAC
:1016500014C0E82FE695E695E695EE31F8F4F0E053
:10166000E856FE4F877021E030E001C0220F8A95D6
:10167000EAF78281822B82830895AAE9B1E0EFEF35
:1016800090E02D91821751F0EF3F19F4211101C024
:10169000E92F9F5F9630A9F7EF3F09F408950E2ECA
:1016A000000CFF0BE856FE4FE6CF80911A02909196
:1016B000E901981301C008958F5F8770FACF292F31
:1016C0009C3078F5893068F590E039E0239F800DF3
:1016D000911D1124682F677023E0969587952A95B0
:1016E000E1F7FC01EE0FFF1FE80FF91FE754FE4F73
:1016F00050E040E080E0219130E0062E02C03695B7
:1017000027950A94E2F721703327042E01C0220F97
:101710000A94EAF7822B4F5F5F4F4330510559F728
:10172000089580E00895292F9C3098F5893088F538
:1017300090E039E0239F800D911D1124282F277000
:1017400041E001C0440F2A95EAF723E0969587957A
:101750002A95E1F7FC01EE0FFF1FE80FF91FE75490
:10176000FE4F30E020E070E05191DF011197CB0196
:10177000022E02C0969587950A94E2F781708195B2
:101780008527842385278C932F5F3F4F2330310596
:1017900059F70895809580FF08C0469A81FF07C0D9
:1017A000479A82FF06C02D9A08954698F7CF47982A
:1017B000F8CF2D9808958093F1027093F30260930F
:1017C000F202809119038430F9F48093E9008FEFDD
:1017D0009091E800815095FD06C095ED9A95F1F73E
:1017E00000008111F5CF8091E80085FF0DC050E029
:1017F00040E063E070E081EF92E00E94D1048091CC
:10180000E8008E778093E8000895BC0184E00E9490
:10181000DB0B0895BC0183E00E94DB0B08959C0163
:1018200084E08093E9009FEF8091E800915085FD6E
:1018300006C085ED8A95F1F700009111F5CF8091F2
:10184000E80085FF0CC050E040E066E070E0C901B0
:101850000E94D1048091E8008E778093E80008957B
:10186000CF93DF93EC0180911A018823B1F180912D
:10187000EF0287FF32C060E284E08093E9008FEFDF
:101880009091E800815095FD06C095ED9A95F1F78D
:1018900000008111F5CF8091E80085FF1BC0809189
:1018A0001A0170E050E040E0811104C050E040E0D7
:1018B00068E070E0CE010E94D1048091E8008E774C
:1018C0008093E80080E2FE01A7EFB2E001900D9264
:1018D0008A95E1F7DF91CF91089568E081E0CDCF5F
:1018E00081E08093E00080E28093D8001092C900EC
:1018F0008FE19EE40197F1F700C0000087E090EBD4
:10190000DC018093270390932803A0932903B093CD
:101910002A0388E19CE00FB6F894A89580936000B4
:101920000FBE90936000FFCF8091DE0280FD0AC061
:10193000E8EAF2E0118210821282339652E0EE3D24
:10194000F507C1F76A9A3EB13B7F2EB124604FB7CD
:10195000F89488EA92E0FC015191CF0168E02EB939
:10196000000000C057FF3EB9550F000000C000C086
:1019700000C03EB900C06A9591F7F2E08E3D9F0726
:1019800051F74FBF8FE594E00197F1F700C00000D9
:101990000895EF92FF920F931F93CF93DF938C01E3
:1019A000C8EAD2E0F12CE12CF80194816091E002C8
:1019B0008091DF02F9E0EF16F104ECF49923E9F0ED
:1019C0009E014091E1020E942E072FEFE21AF20AD7
:1019D000239682E1E816F10439F70E94940CF8018D
:1019E000848190E00196817099278483CDB7DEB71A
:1019F000E6E00C94052A992319F39E0140E0E3CF19
:101A0000B0E0A0E0E6E0FDE00C94E329EC014C81BD
:101A1000042F10E09801D8010E94B4299B01AC0169
:101A20000E94CA294B015C01E0E2F0E0E01BF10BEF
:101A3000A5E5B0E0AC019B010E94CA296B017C01C5
:101A40009F01DF010E94AC299B01AC010E94D529B6
:101A50009B01AC01280D391D4A1D5B1DC701B60154
:101A60000E947D29F22E822F90E039E23F1598F1F5
:101A700043E0249F9001112435952795122F10954E
:101A800098EAC92E92E0D92E00E085E5E82EEF18FD
:101A90008E2D01FD8F2D9601412F6091E0020E9455
:101AA0002E070F5F53E0C50ED11C023189F70E944B
:101AB000940C9C8181E0992319F0903219F48FEFF6
:101AC0008093190180911901890F8C83CDB7DEB7FE
:101AD000ECE00C94FF2925E530E0A901481B590BE7
:101AE000CA019A01220F331F280F391F37FFC4CFB5
:101AF0002F5F3F4FC1CF0F931F93CF93DF93C8EA60
:101B0000D2E0FE01118210821282339682E0EE3D15
:101B1000F807C1F710E000E08091A602082E000C43
:101B2000990B081719078CF180911801082E000CE9
:101B3000990B801791074CF19E014091E102609151
:101B4000E0028091DF020E942E070F5F1F4F239655
:101B50000231110509F70E94940C809117019091B0
:101B6000A602980F9093A60220911801280F2093A7
:101B70001801121614F491311CF08195809317010D
:101B8000DF91CF911F910F910895198218821A82C7
:101B9000DCCFB0E0A0E0EFECFDE00C94E629FC0126
:101BA0008281DD24DA9480FD02C0DD24D39408EA2A
:101BB00012E0D0E0C0E022E1B22EF80111821082E2
:101BC000128294E0E92EF12CC12C8091A5028C0D9B
:101BD0008331C4F16B2D0E944729892F082E000CF8
:101BE000990B8C179D0791F48091E1028E9DA001C5
:101BF0008F9D500D11245595479555954795980102
:101C00006091E0028091DF020E942E07CD0CF1E08E
:101C1000EF1AF108D1F621960D5F1F4FC231D105A1
:101C200061F60E94940C8091A50291E0D91210C037
:101C300081110CC081E18093A502CDB7DEB7E9E048
:101C40000C94022A87FFCACF8E5EC8CF8150F3CF93
:101C500090E00196BE010E946929EDCFEF92FF92BC
:101C60001F93CF93DF93EC0188EAE82E82E0F82EF1
:101C700010E08C8197014091E1026091E002810FB8
:101C80000E942E07125F83E0E80EF11C1C3F89F7CB
:101C90000E94940C9A818C8190FF08C08F5F8C8386
:101CA000DF91CF911F91FF90EF9008958150F7CF72
:101CB0009091DE0290FF0CC0E8EAF2E0818360833D
:101CC0004283339692E0EE3DF907C1F70E94940CEF
:101CD0000895A3E0B0E0EFE6FEE00C94EB298C0160
:101CE0008091A70281110AC09E012F5F3F4F4FEFE5
:101CF0006FEF0E942E078A818093A702F80164810A
:101D0000613069F08091A70240E0662361F040E015
:101D1000623011F44091A70280E060E004C060915D
:101D2000A70240E080E00E94580EF801848190E014
:101D3000019663E070E00E94692984832396E4E0C1
:101D40000C94072AA3E0B0E0E8EAFEE00C94ED2949
:101D50009091DE0290FF0AC09E012F5F3F4F0E94CC
:101D60002E074B8169818A810E94580E2396E2E0FA
:101D70000C94092ACF93DF93EC01EEEDF2E043815E
:101D800062818C810E94A20E8C818F5F8C83DF9197
:101D9000CF910895CF93DF93EC01EC81F0E0E5570C
:101DA000FC4F4491EEEDF2E0628181810E94A20E2F
:101DB0008C818F5F8C83DF91CF910895CF93DF93D8
:101DC000C7E8D3E060E0CE010E94342A2196C11515
:101DD00084E0D807B9F7DF91CF9108951F93CF938F
:101DE000DF93122F8430E0F46C30D0F44930C0F42B
:101DF000C42FD0E0CC0FDD1F92E1699FC00DD11D33
:101E0000112498ED899FC00DD11D1124632FCE019F
:101E100087960E94342A612FCE0188960E94342A28
:101E2000DF91CF911F910895AF92BF92CF92DF9231
:101E3000EF92FF921F93CF93DF938BE8C82E84E03D
:101E4000D82ED0E07601C0E014C0F5012591349180
:101E5000412F6C2F8D2F0E94EE0E82E0A80EB11C38
:101E60001F5F193091F782E1E80EF11CCF5FCC3093
:101E700019F0570110E0E9CFDF5F88EDC80ED11CE3
:101E8000D43001F7DF91CF911F91FF90EF90DF9059
:101E9000CF90BF90AF900895CF93C82F6FEF81116F
:101EA00062E283E290E00E94342A6FEFC11161E1A7
:101EB00084E290E00E94342A6FEFC11165E085E270
:101EC00090E00E94342ACF91089580E00E944C0F48
:101ED00060E086E290E00E94342A0E94140F0E9483
:101EE000DE0E81E00E944C0F0895682F86E090E09E
:101EF0000E94342A08950F931F93CF93DF93843069
:101F000030F56C3020F5493010F5C42FD0E0CC0FFF
:101F1000DD1F22E1629FC00DD11D112438ED839F8A
:101F2000C00DD11D1124CE0187960E94202A082FB2
:101F300010E0102F0027CE0188960E94202A9801D9
:101F4000282BC901DF91CF911F910F91089590E047
:101F500080E0F8CF462F843040F47C3030F4693094
:101F600020F4672F0E947B0F089590E080E0089591
:101F7000CF92DF92FF920F931F93CF93DF936C0169
:101F80000091260380913F02082BC7E0D0E010E0CB
:101F9000FC2EC8010C2E02C0959587950A94E2F795
:101FA00080FD0CC02197A0F7F12C8F2DDF91CF91F0
:101FB0001F910F91FF90DF90CF900895B6018C2F65
:101FC0000E94AA0F0E945C09019761F3EECFCF93A4
:101FD000DF93EC010E94B80FBE010E94AA0F0E947D
:101FE0005C09DF91CF910895FC0183819481892B55
:101FF00029F08081918189238F3F51F480E00895F9
:10200000843FE1F717C0883EA8F0813FB9F712C0BE
:10201000808191810E94E70F92959F70963099F38D
:1020200058F4925F9F70923048F7803F19F040F764
:10203000883E20F781E008959A5FF4CF83E290E034
:102040000E94202A823289F484E290E00E94202AB1
:10205000813159F485E290E00E94202A91E0853098
:1020600009F090E0892F8170089580E0FCCFCF9334
:1020700084E090E00E94202AC82F82E290E00E9433
:10208000202A982F8C2FCF910895CF92DF92EF9234
:10209000FF926B017C010E941F07B701A60188E037
:1020A00090E00E94462AFF90EF90DF90CF90089535
:1020B000A3E0B0E0EEE5F0E10C94E029F82E762EF6
:1020C000E42E622E9091DE0290FF29C0E92FE69562
:1020D000AE2FB0E0AF59BE4F8C918093A3029E7F8C
:1020E000923009F59E012F5F3F4F8F2D0E942E07E2
:1020F0004B8169818A810E94580EF092DF027092B2
:10210000E002E092E102662051F06091DE027091FF
:10211000DF028091E0029091E1020E944510239637
:10212000EFE00C94FC29823019F4E090E102E5CF55
:10213000863019F4F090DF02E0CF8930D9F389318D
:10214000E1F6E9518E2F8170582EE695F0E0EA57BE
:10215000FC4FE4910E2F10E088EAC82E82E0D82EC2
:10216000B12CA12C92E1892E912CC501B4010E94C1
:1021700055298F2D511013C0860F96014E2D672DB6
:102180000E942E07A00EB11E83E0C80ED11C8EED5A
:10219000C81682E0D80649F70E94940CAECF861B81
:1021A000ECCFEEEDF2E0438128E0421B08F440E082
:1021B00021E0628181810E9458100895EEEDF2E0E5
:1021C000438128E0420F08F44FEF21E062818181D2
:1021D0000E9458100895EEEDF2E0628128E0621B43
:1021E00008F460E021E0438181810E945810089545
:1021F000EEEDF2E0628128E0620F08F46FEF21E07B
:10220000438181810E9458100895EEEDF2E08181B2
:1022100021E04381628188500E9458100895EEEDBC
:10222000F2E0818121E043816281885F0E94581041
:1022300008958091E202882319F081508093E20290
:102240006091DE027091DF028091E0029091E102E4
:102250000E94451008958091E202833018F48F5F48
:102260008093E2026091DE027091DF028091E002D1
:102270009091E1020E94451008959091DE0290FF36
:102280002CC0917081112AC092609093DE02662367
:1022900051F06091DE027091DF028091E002909136
:1022A000E1020E9445106091DE02669570E04BE00D
:1022B00050E08CE091E00E94682A892BB1F01092E6
:1022C000A40281E08093A00220E04091E1026091AD
:1022D000E0028091DF020E9458100895853210F0CC
:1022E0009864D3CF880F982BD0CF81E08093A4023D
:1022F0000E94180690939E0280939D02E2CF8091E7
:10230000DE028695815009F484E261E00E943D116D
:1023100008958091DE0286958F5F853208F081E016
:1023200061E00E943D1108959091DE0290FF08C087
:102330009695981728F0961718F40E948911089519
:1023400061E00E943D110895EEEDF2E083E08083AC
:1023500011828FEF828383831482608171818281F5
:1023600093810E944510089580913D0290913C0216
:10237000892B8093980190913E029923A1F0892B9B
:102380008093980180911A018823E1F18091EF02F6
:1023900087FF38C08EE1EAE9F1E090E08150A0F5D6
:1023A00091110E94E90A40E250E06CE172E088E994
:1023B00091E00E94752A892B21F180E2E8E9F1E0A1
:1023C000ACE1B2E001900D928A95E1F7E091E6026E
:1023D000F091E7023097A9F080911A01882359F013
:1023E0008091EF0287FF07C0809198018093990147
:1023F00086E0809398010280F381E02D88E991E0E6
:102400000995089586E0C7CF2191222339F29F5F75
:10241000C5CF90E080E00E943A0690E080E00E9404
:10242000240610923C020E94B41186E0E7E9F2E033
:10243000DF011D928A95E9F71092910210929002A5
:10244000109292020E94C4070895809326030E946E
:102450000912089580912603982F9670963021F4E2
:1024600088600E9425120895877FFBCF21E030E02D
:1024700001C0220F8A95EAF72095809126038223D6
:102480000E942512089590911B02809589238093C4
:102490001B02282F277091F4282F082E000C330BD5
:1024A0009217130659F09091F00292FF07C085959C
:1024B000859585950E94361210921B020895CF9340
:1024C000C091F002C2FB992790F9981791F080FB18
:1024D000C2F9C093F0026091EF0284E090E00E94A4
:1024E000342A6C2F82E290E00E94342A82E00E941B
:1024F0004312CF91089521E030E001C0220F8A9568
:10250000EAF780912603822B0E942512089580937A
:102510003F020E9409120895882321F00E94EF0AC9
:102520000E94B4110895882339F090913D02982BB0
:1025300090933D020E94B4110895882309F455C078
:10254000823879F40E94500681FF4FC089E30E94CF
:10255000210B0E94B41189E30E94F60A0E94B41173
:102560000895833859F40E94500680FF3EC083E5E9
:102570000E94210B0E94B41183E5EECF843859F4F8
:102580000E94500682FF31C087E40E94210B0E9406
:10259000B41187E4E1CF9CEF980F913AE8F290E212
:1025A000980F983050F4877091E001C0990F8A9588
:1025B000EAF7892F0E94EF0AD1CF9BE5980F93305D
:1025C00028F490E080E00E943A06089598E5980F7C
:1025D000973128F490E080E00E9424060895803F1F
:1025E00020F00E94EB070E94C4070895CF93C82FE4
:1025F0008823C9F08238C9F40E94500681FD13C0B7
:1026000089E30E94210B0E94B4112FEF87EE93E023
:10261000215080409040E1F700C0000089E30E9413
:10262000F60A0E94B411CF9108958338A1F40E9454
:10263000500680FDF8CF83E50E94210B0E94B41163
:102640002FEF81EE94E0215080409040E1F700C0F0
:10265000000083E5E4CF8438A1F40E94500682FD97
:10266000E2CF87E40E94210B0E94B4112FEF81EE8C
:1026700094E0215080409040E1F700C0000087E4E2
:10268000CECF8CEF8C0F813A88F580911A01882388
:1026900001F18091EF0287FF1CC0EC2FE695E695D3
:1026A000E695F0E0E856FE4F828190E04C2F4770AF
:1026B00021E030E002C0220F331F4A95E2F7822367
:1026C0009323892B79F08C2F0E94F60A0E94B41173
:1026D00009C0EAE9F1E08191C817A9F321E0E03AE5
:1026E000F207C9F78C2F0E94210B9BCF80E28C0F41
:1026F000883068F4C77021E030E001C0220FCA952D
:10270000EAF780913D02822B80933D028ACFEBE570
:10271000EC0FE33040F4F0E0E55EFE4F808190E0A6
:102720000E943A0680CFE8E5EC0FE73150F4F0E084
:10273000EE0FFF1FE25EFE4F808191810E94240612
:1027400072CFC03F08F46FCF8C2F0E94A6080E9462
:10275000C40769CF1F93CF93DF93182FD0E0C0E059
:10276000893311F4C0E5D0E0812F0E94F612209742
:1027700039F4812F0E949D12DF91CF911F9108950E
:102780008FE99FE00197F1F700C000002197EFCF9C
:102790000F931F93CF93DF93C62FD42F022FFC01EB
:1027A00082818823A9F0609325030E9418069093E4
:1027B000240380932303C77081E001C0880FCA956A
:1027C000EAF70E949312DF91CF911F910F91089524
:1027D00080912503681332C08091230390912403D4
:1027E0000E940906883C910548F510E21D0FCD179F
:1027F000B9F080E28C0F883040F4C77081E001C0EE
:10280000880FCA95EAF70E948C12183048F481E0CC
:102810009D2F977001C0880F9A95EAF70E94931236
:10282000802F0E94AA13183070F6D77081E001C083
:10283000880FDA95EAF70E948C12C5CFC77081E045
:1028400001C0880FCA95EAF7F6CF68EE7EEF90E0F8
:1028500080E00E94522A60E082E090E00E94342AE8
:1028600060E083E090E00E94342A10923F0260E032
:1028700084E090E00E94342A64E082E290E00E94CA
:10288000342A60E085E090E00E94342A60E086E02F
:1028900090E00E94342A6FEF87E090E00E94342A93
:1028A00040E050E0BA0188E090E00E94462A60E0F3
:1028B0008DE090E00E94342A40E050E0BA0188E1C7
:1028C00090E00E94462A60E087E190E00E94342A6E
:1028D00040E050E0BA018CE190E00E94462A70E0AE
:1028E00060E080E290E00E94522A40E050E0BA01AD
:1028F00088E190E00E94462A80E00E944C0F0E94EE
:10290000650F40E050E0BA018FE090E00E94462A57
:1029100040E050E0BA0183E190E00E94462A089529
:1029200010923D0280911A01EAE9F1E0882361F0FA
:102930008091EF0287FF08C08EE1DF011D928A952A
:10294000E9F70E940912089586E0F7CFAAE2B0E005
:10295000ECEAF4E10C94EC298BE193E02091F10096
:10296000DC012D93CD01B3E083329B07B9F7809151
:102970001C03833009F472C0B8F4813009F449C0F3
:10298000823009F4B3C08091E80083FF8BC280914C
:102990001B0390911C039A3008F084C2E92FF0E0E9
:1029A000EC57F54D0C949F298A3009F48EC08B307A
:1029B00009F471C0893039F780911B03813219F70E
:1029C00080911F0390912003009711F00297D9F690
:1029D0008091E800877F8093E8008091E80082FF83
:1029E00038C09091F3008091F200029731F4809109
:1029F000F100813011F0863021F48091F100809354
:102A0000F6028091E8008B778093E8000E94FB0437
:102A1000BACF80911B03813A09F0B5CF8091E800CD
:102A2000877F8093E80080911F0390912003892B7A
:102A300061F460E287EF92E070E00E94A705809168
:102A4000E8008B778093E8009ECF60E090E080E024
:102A5000F3CF809119038111C0CF95CF80911B03D3
:102A6000813A09F090CF80911F0390912003892B28
:102A700009F089CF8091E800877F8093E8008091FA
:102A8000E80080FFFCCF80911A018093F1008091D3
:102A9000E8008E77B9CF80911B03813209F073CFA4
:102AA00080911F0390912003892B09F06CCF8091B6
:102AB000E800877F8093E8000E94FB0480911D035B
:102AC00080931A010E9490145ECF80911B03813283
:102AD00009F059CF8091E800877F8093E8000E9439
:102AE000FB0480911E038093F5024DCF80911B0360
:102AF000813A09F048CF8091E800877F8093E80011
:102B00008091E80080FFFCCF8091F502BECF803835
:102B100099F0823809F0C6C180911F038F70873009
:102B200008F0C0C18093E9008091EB0085FB882705
:102B300080F91092E90006C0809117039091180364
:102B4000911182609091E800977F9093E8008093C4
:102B5000F1001092F1008091E8008E779FC18823E8
:102B600009F48DC1823009F09DC180911D0381114E
:102B700090C180911F038F702FEF280F263008F02F
:102B800091C18093E9002091EB0020FF82C1933036
:102B900031F48091EB0080628093EB007AC19091D8
:102BA000EB0090619093EB0021E030E001C0220F38
:102BB0008A95EAF72093EA001092EA008091EB00F0
:102BC0008860EACF81116EC110911D031F7780913B
:102BD000E3008078812B8093E3008091E800877F79
:102BE0008093E8000E94FB048091E80080FFFCCF06
:102BF0008091E30080688093E30082E0111183E01C
:102C0000809319034FC18058823008F04BC1209146
:102C10001D0330911E032C3DE3E03E07A1F583E048
:102C20008A838AE289834FB7F894DE01139620E005
:102C30003EE051E2E32FF0E050935700E49120FF93
:102C400003C0E295EF703F5FEF708E2F90E0EA30A7
:102C5000C0F0C7968D939D932F5F243159F74FBFD6
:102C60008091E800877F8093E8006AE270E0CE01FF
:102C700001960E94A7058091E8008B778093E80079
:102C800011C1C096E7CF80911F0390912003432F7D
:102C900055274330510509F44AC078F541305105B4
:102CA00009F47AC08BE590E0EBEEF7E04230510595
:102CB00009F0F8C02091E800277F2093E8002091D8
:102CC0002103309122038217930708F49C0140E00E
:102CD0002115310509F065C0411163C08091E800FC
:102CE00082FDC9CF80911903882329F2853019F21A
:102CF0008091E80083FFF2CFBECF4132510509F445
:102D00003CC04232510509F0CDC08330910508F036
:102D1000C9C0FC01EE0FFF1FE757FE4F0190F08185
:102D2000E02D8A579E4FDC018C9190E01AC033272A
:102D300021303105D1F02115310561F02230310506
:102D400009F0B0C0E8E5F8E0E4918E2F90E0E8E506
:102D5000F8E007C0EAE8F8E0E4918E2F90E0EAE8B6
:102D6000F8E0009709F49EC0A5CFEEE7F8E0E49103
:102D70008E2F90E0EEE7F8E0F4CF8330910508F075
:102D800091C0880F991FFC01E157FE4F0190F0811F
:102D9000E02D89E090E08ECF82E190E0E6E4F8E07B
:102DA00089CF80911903882309F465CF853009F410
:102DB00062CF8091E80083FD5ECF8091E80082FDC4
:102DC0008DCF8091E80080FF83CF9091F3008091B8
:102DD000F2002115310519F08830910550F041E0DD
:102DE000089709F040E08091E8008E778093E80032
:102DF0006FCF44914093F1003196215031090196F3
:102E0000E8CF803809F04EC08091E800877F80933A
:102E1000E80080911A038093F1009DCE811142C099
:102E200010911D031230F0F58091E800877F8093A8
:102E3000E80010931A030E94FB04112311F084E0B0
:102E400005C08091E30087FDFACF81E080931903EC
:102E500042E061EC81E00E941A0542E261EC84E00C
:102E60000E941A0542E261EC82E00E941A0542E2E9
:102E700060EC83E00E941A058091190313C08091D1
:102E80001D03813079F481E0933009F080E0809374
:102E900018031092E9008091E800877F8093E80092
:102EA0000E94FB048091E80083FF0AC08091E80043
:102EB000877F8093E8008091EB0080628093EB0035
:102EC000AA96E3E00C94082A0E9490142FEF84E362
:102ED0009CE0215080409040E1F700C0000088E174
:102EE0009CE00FB6F894A895809360000FBE909375
:102EF0006000FFCFA5E0B0E0E0E8F7E10C94DE2948
:102F00008C01FC0183819481892B31F08081918136
:102F100089238F3F09F062C62596E1E10C94FA29D6
:102F20000E94B80FF82E682F89819A810E94930B16
:102F300069817A818F2D0E94AA0F7C01F80182811C
:102F4000882309F41EC6C70182519F45409708F0A7
:102F50008BC58FEF93E00E94202A811128C0FEEEDE
:102F6000EF0E57E8852E53E0952EE11032C01C82FB
:102F70001B82442443944AE0342E74018FEFE81AF4
:102F8000F80AC4010E94202A89831A82882379F0D2
:102F90009FEF980F933058F58A83498292E0890E0B
:102FA000911CC7010E94202A8B83811121C080912E
:102FB0001B02877009F4B0CFF8018281882309F4DD
:102FC000ABCF8091F00282FFA7CF82E00E94431234
:102FD000A3CF811424E0920651F3C4010E94202A59
:102FE000811101C0EA943FEF831A930ABECF4701D3
:102FF000FE0131967F01F7012081222309F4BDCF24
:10300000213009F047C091818281913031F4F2E0A2
:10301000EF0EF11C0E94AA1307C0923049F422E07F
:10302000E20EF11C0E94F6123FEFE31AF30AE3CF1F
:10303000933031F432E0E30EF11C0E949D12F4CF84
:10304000943021F08FEFE81AF80AEECF92E0E90E03
:10305000F11C30E020E0B7016F5F7F4FF701418145
:103060008053990B8A30910550F021503109E0F2DC
:103070008FE99FE00197F1F700C00000F6CF329E84
:10308000F001339EF00D11249C012E0F3F1F842F61
:103090007B01E1CFE22FF0E0EC50FE4F5490822F05
:1030A00086958695869590E0FC01EC51FE4F6490E4
:1030B0002770712C022E02C0759467940A94E2F76F
:1030C000E1E06E227724FC01EC52FE4FA490B12C7B
:1030D000022E02C0B594A7940A94E2F7F1E0AF2261
:1030E000BB24FC01EC53FE4FC490D12C02C0D594FC
:1030F000C7942A95E2F721E0C222DD24611471040D
:1031000019F081EE0E94F612A114B10419F086EEB6
:103110000E94F612852D0E94AA13A114B10419F081
:1031200086EE0E949D126114710419F081EE0E94D6
:103130009D12C114D10409F477CF8CE26BCF81E0EA
:103140000E947B1203C081E00E9436120E942A1264
:103150002ECF82E0F5CF82E0F7CF2FEBE2162CE501
:10316000F20609F44BC0A0F180ECE8168CE5F806F5
:1031700009F09BC49091E302892F869586958695E8
:103180008F5F8F719770863008F059C0880F880F55
:10319000880F892B8093E3028091E30210C085E0C1
:1031A0000E9401078091E3020E94750F00CF809179
:1031B000E302982F987FE9F188508093E302887F9B
:1031C00091E009F490E08091E30290FB80F913C054
:1031D0008091E302982F969596959695953040F4B8
:1031E0009F5F990F990F990F8770892B8093E30246
:1031F0008091E30281608093E30219C08091E30231
:1032000080FF09C08E7F8093E3020E94750F80E0EB
:103210000E945D06CCCE80FDCACE81608093E30221
:10322000813019F489E08093E3028091E3020E94E7
:10323000750F8091E302869586958695E9CF9093E8
:10324000E302AACF27E245EE65EEC4C426E241EED2
:1032500060EEC0C427E245EE64EEBCC426E241EE57
:1032600062EEB8C428E241E0EFCFF5EAEF16FDE5E3
:10327000FF0609F447C4E0F431E6E3163DE5F30642
:1032800009F440C426E1E2162CE5F20609F0B7C4C1
:1032900080913D028A7A91E009F490E09093B80120
:1032A00081113FC189E20E94210B0E94B4117FCE9F
:1032B000C7018D5A9D45039728F724C48091EF02DA
:1032C0008062F7E0EF16FCE5FF0609F4B1C08091DB
:1032D000EF02806128E0E2162CE5F20608F4A8C0AF
:1032E0008091EF028064A4C03DE0E3163CE5F30664
:1032F00009F4D5C0B0F48091EF028E7F9BE0E9160F
:103300009CE5F90609F494C08091EF028C60ECE032
:10331000EE16ECE5FE0608F48BC08091EF028D7F7F
:1033200087C0FFE0EF16FCE5FF0609F4C8C008F40B
:10333000BAC030E1E3163CE5F30609F4C4C081E10C
:10334000E8168CE5F80609F00CC48091EF028F7B3B
:103350006FC09FEFE9169CE5F90609F4C2C0D8F5E5
:10336000FAEFEF16FCE5FF0609F487C0D0F434E16C
:10337000E3163CE5F30609F4C2C008F4AEC095E1DB
:10338000E9169CE5F90609F0ECC38091EF0282FB97
:10339000992790F921E0922790FB82F990FB83F91D
:1033A00047C0ECEFEE16ECE5FE0609F480C008F429
:1033B00068C02DEFE2162CE5F20609F47CC080917E
:1033C000F00283603EEFE3163CE5F30609F0C9C363
:1033D0008093F002C6C381E6E8168DE5F80609F48D
:1033E00099C0A0F4E1E0EE16EDE5FE0609F490C008
:1033F00008F47BC060E022E0E2162DE5F20609F059
:10340000B0C38EE090E00E94342AABC33DEAE316DD
:103410003DE5F30611F178F49091EF02892F8E7F4C
:1034200090FF816095EAE9169DE5F90609F099C3D8
:103430008093EF0296C3EEEAEE16EDE5FE0659F133
:10344000FFEAEF16FDE5FF0609F08BC39091F0024D
:10345000892F877F93FF8860BBCF8091F0028860BF
:10346000B7CF8091EF028260E3CF8091EF0284605A
:10347000DFCF8091EF028860DBCF8091F002816026
:10348000A7CF8091F0028260A3CF0E949014809118
:10349000EF028068CDCF8091F002877F99CF809135
:1034A000EF028B7FC5CF8091EF02877FC1CF8091E4
:1034B000F0028E7F8DCF8091F0028D7F89CF809139
:1034C000EF028F7EB5CF8091EF028F7DB1CF0E944A
:1034D00090148091EF028F77ABCF8091EF02837FC2
:1034E000A7CF8091F0028C7F73CF8091F002982F4C
:1034F000909591708E7F892B90FB81F969CF0E9406
:1035000090149091EF02892F97FB87F9805890CF04
:1035100061E077CF9091EF02892F8F7E94FF8061D9
:1035200087CF85E3C0CE85E35EC481608093DE02F1
:1035300061E086950E943D113ACD4FE751E169E87F
:1035400071E10E94180733CD49E851E16FE771E15D
:10355000F8CF4FE051E165E071E1F3CF4BEE50E180
:1035600068EF70E1EECF41ED50E16EED70E1E9CF33
:103570004EED50E161ED70E1E4CF4BE251E169E1E4
:1035800071E1DFCF61E081E0D5CF65E082E00E94AC
:1035900094110DCD68E086E0FACF64E18FE0F7CFBB
:1035A00067E185E1F4CF62E289E1F1CF61E083E296
:1035B000C1CF0E949014EFEFF4E32CE0E150F04013
:1035C0002040E1F700C000000E94700C8091F002E2
:1035D00082FB882780F991E089270E945F12F80119
:1035E0008281E080F180882309F445C0C7010E94F0
:1035F000B80FD82E682FC7010E94930BB7018D2DED
:103600000E94AA0F0E945C097C01882EF801D280DA
:10361000B580B2943FE0B32280911B028770C1F065
:10362000AD2CDD20B1F08F2D807F803421F080E241
:103630008E0D883068F08091F00282FF09C082E030
:103640000E94431280911B028770AA24A3948111C7
:10365000A12C9F2C92942FE09222FBE0F91508F404
:1036600079C0E92DF0E0E257F54D0C949F2981E0F7
:10367000B4CF80E0B2CFC7010E945F0BD82EBECF7F
:103680002F2D2F70C22E8F2D807F19F0C29490EFB6
:10369000C922DD20B9F0CC2069F080E28E0D88309F
:1036A00010F0811009C080913D02C82AC0923D02ED
:1036B0000E94B4118E2D4CC080913C02C82AC09249
:1036C0003C02F6CF8E2D0E949D12CC2009F442C000
:1036D00080E28E0D883010F0811004C08C2D0E9485
:1036E000EF0A06C0C09480913C02C822C0923C02FE
:1036F0000E94B4112FC03F2D3F70C32E8F2D807FAD
:10370000803219F0C29480EFC822882089F081E0CD
:10371000881609F46AC0DD2009F474C0BB2009F4DE
:103720006AC0F801858180FFC5CF8F70858363C033
:103730002091F00222FD37C0DD2079F1CC2039F054
:1037400080913D02C82AC0923D020E94B41180E0DF
:103750000E94F612292D2850330B2430310520F415
:103760000E9450060E94CA0BAA2009F4D5CB809172
:103770001B0280FDD1CBF801128285958595859538
:103780000E947B12C8010E947A1780911B028595C6
:10379000859585950E943612BFCB80E00E949D12D0
:1037A000CC20C1F29BCFDD2099F090913E028C2D70
:1037B000892BB11003C00E949312CCCFE1E0BE125E
:1037C000FACF22FFC7CF981729F280933E02C2CFCB
:1037D000B11006C00E94E90A8C2D0E948C12BACF4B
:1037E000F1E0BF1609F4B6CFF5CFDD2031F025E0CA
:1037F0002B1508F4AFCF8C2DDECF34E03B1508F449
:10380000A9CFEACFBB2041F3F9E38F1209C02FEF14
:1038100037EE83E0215030408040E1F700C00000E7
:103820008E2D0E949D1296CF8F2D86958695837042
:1038300061F0813009F08ECFC7019370D11002C0C2
:1038400090E080E00E94240685CFC7019370D110DC
:1038500002C090E080E00E943A067CCF8E2DDD20F1
:1038600029F00E94A6080E94C40774CF0E94EB07AB
:10387000FACF8F2D837091F5D1106CCF4E2D4295DC
:1038800046954770440F440F8E2D8F70042E01C053
:10389000880F0A94EAF72E2D2071E4FE07C02FE06E
:1038A00030E001C0220F4A95EAF720953F2D36956A
:1038B00036953370323069F050F440913F02313028
:1038C00029F0822B84230E94871244CF842B822BE1
:1038D000FACF282B80913F028227F5CF8695DD20F5
:1038E00011F08F2D8170882309F434CF4E2D42952D
:1038F00046954770440F440F8E2D8F70042E01C0E3
:10390000880F0A94EAF72E2D2071E4FE07C02FE0FD
:1039100030E001C0220F4A95EAF720953F2D3695F9
:1039200036953370323069F050F4409126033130CF
:1039300029F0822B84230E9425120CCF842B822B0A
:10394000FACF282B809126038227F5CF9F2D9F70D9
:10395000F92EDD2029F0892F0E947B128E2D2BCF8E
:103960008E2D0E948C128F2D0E943612F3CE8E2D3A
:10397000E2EF8E16B1F1E81570F0F0EF8F16D1F08E
:1039800021EF821691F0DD2009F45EC0B11092CED5
:103990008F2D8F712AC033EF831651F194EF891266
:1039A000F2CF8091F00282FD2FC08F2D8F71DD202C
:1039B000D9F21BC0DD2081F0E4E0EB1508F4CACE9B
:1039C0002F2D2F7181E090E001C0880F2A95EAF732
:1039D000909126038927AFCFF5E0FB1508F4BACE06
:1039E000EFCF8F2D8F71D110BFCF0E947B12B2CE3F
:1039F00080E0DD2009F49FCF9F2D9F7181E001C001
:103A0000880F9A95EAF797CFDD2099F02F2D2F7127
:103A1000F22E822F0E947B128091F00282FF07C05B
:103A200038E0F39EC0011124836080931B028F2D28
:103A3000DCCF81E00E94431281E08B1508F08ACE32
:103A400082E00E94431286CEBB2059F0893309F0F0
:103A5000E7CE9FEFE7EEF3E09150E040F040E1F772
:103A6000DDCE8F2D8F7180CFF0E1EF16FFE5FF06E1
:103A700009F465CB21E1E2162FE5F20609F469CBE2
:103A80008DEBE8168CE5F80609F491CB08F065CBD0
:103A9000EBEBEE16ECE5FE0609F481CB80E0FCEBE7
:103AA000EF16FCE5FF0609F47BCB83EFE8168CE507
:103AB000F80609F4CBCB08F099C1E8EDEE16ECE579
:103AC000FE0609F4BFCBF9EDEF16FCE5FF0609F49D
:103AD000C9CB27EDE2162CE5F20609F478C0109266
:103AE000250393E0E9169DE5F90608F0BECBEAEF61
:103AF000EE16ECE5FE0630F4C70182509C45449773
:103B000008F0C0CB0E9437109093F0028093EF0230
:103B100082E1E8168CE5F80609F4D9CC08F019CC56
:103B2000E9E0EE16ECE5FE0609F4AFCC08F0DCCBDC
:103B300025E0E2162CE5F20609F49BCC08F0BECB9A
:103B400083E0E8168CE5F80609F48BCC08F08DCC00
:103B50008091EF028160E2E0EE16ECE5FE0609F4EA
:103B600067CC6091EF02F090F00284E090E00E9458
:103B7000342A6F2D82E290E00E94342A0E94901431
:103B800016CA30E1E3163FE5F30609F4DCCA81E129
:103B9000E8168FE5F80609F4DECA23EFE2162CE5F5
:103BA000F20609F453CB08F006C188EDE8168CE55F
:103BB000F80609F447CB99EDE9169CE5F90609F4F6
:103BC00051CBE7EDEE16ECE5FE0609F001C126E269
:103BD00041EE61EEC8010E94C813E9C985E0DE012B
:103BE000119601900D928A95E1F7F8012281898161
:103BF0009A81211195C90E945F0BF82E99C92AE577
:103C0000E2162DE5F20609F432CD78F4E1148CE5E4
:103C1000F80609F4CECC9EEDE9169CE5F90609F00C
:103C2000DECC0E9425140E946417ECE5EE16EDE54B
:103C3000FE0609F4CBCC08F41CCD27EAE2162DE5EC
:103C4000F20689F3CCCC80913D0282723CECE31603
:103C50003CE5F30609F491CC08F06DC0E6ECEE16F5
:103C6000ECE5FE0609F475CCE8F523ECE2162CE54C
:103C7000F20609F462CC28F582ECE8168CE5F80629
:103C800009F0ADCC8091DE0280FF4FCC8E7F809317
:103C9000DE026091DE027091DF028091E00290917D
:103CA000E1020E9445101092A4023FEF80E792E0EB
:103CB000315080409040E1F700C000000E94940C19
:103CC00076C994ECE9169CE5F90609F43DCC45E08B
:103CD00051E16FE071E1E5ECEE16ECE5FE0609F46A
:103CE00030CC7DCCF9ECEF16FCE5FF0609F43BCCBB
:103CF00088F437ECE3163CE5F30609F42FCC48EFE3
:103D000050E16BEE70E198ECE9169CE5F90609F4D8
:103D100018CC65CCEAECEE16ECE5FE0609F428CCEE
:103D200049E151E16BE271E1FBECEF16FCE5FF06C6
:103D300009F407CC54CC21EDE2162CE5F20609F487
:103D40002CCCB8F48EECE8168CE5F80609F41DCC02
:103D500008F418CCEFECEE16ECE5FE0609F41ACCEC
:103D60006EE089E0F0EDEF16FCE5FF0609F40FCCFC
:103D700036CC24EDE2162CE5F20609F414CC78F4E6
:103D800082EDE8168CE5F80609F40ACC61E088E1DA
:103D900093EDE9169CE5F90609F4CCCB20CCE5EDD2
:103DA000EE16ECE5FE0609F401CCFDE5EF16FF0684
:103DB00009F4FDC814CCF5EFEF16FCE5FF0609F495
:103DC0004DCA08F447CA36EFE3163CE5F306E1F0C6
:103DD000F6E1EF16FCE5FF0609F035CF8091B8015A
:103DE0008111A1CB89E20E94F60A5FCA35EFE31682
:103DF0003CE5F30609F432CA08F42CCA96EFE9163A
:103E00009CE5F90609F06BCE27E245EE66EEE2CEC0
:103E10001F93CF93DF938091E801807F09F049C021
:103E20008091E501882309F444C080911A02D09161
:103E3000E9016091E3017091E401A091E601B09184
:103E4000E701C62FC72316E0D81799F190E0109725
:103E500011F0CF3F19F401968770F6CF189F9001AB
:103E6000199F300D1124F901E651FE4F418147138E
:103E7000F2CF40814613EFCF42814111ECCF438115
:103E800054814A1B5B0B483C510528F78091E8019F
:103E90008F7080618093E801F901E151FE4F8081CC
:103EA0008F708061808383EE91E00E947A170E9478
:103EB000550BDF91CF911F910895A1E1B0E0E3E6AA
:103EC000FFE10C94E5298C0185E0F801DE011D96E7
:103ED00001900D928A95E1F7F801E28083EEA82E19
:103EE00081E0B82E6091E6017091E70161157105DE
:103EF00009F426C19091E3014091E401892F8423C4
:103F00008F3F09F41DC120813181C380D480F0909E
:103F1000E501F601E61BF70BFF2009F4DCC08091F8
:103F2000E801582F507FE83CF10508F09FC051117F
:103F30006BC0FE2C431314C0921312C0E11010C0CA
:103F40008F7080618093E801C5010E947A1780918B
:103F5000E801F80185838F2D6196EAE00C94012A2F
:103F6000C114D10429F0822F83238F3F09F003C1AC
:103F700080E0F82FF170DF2E80FF3CC080911A02A4
:103F80004091E90156E0841315C02D873E878D8549
:103F90009E850E94E70F292F22952F702230F0F086
:103FA000243018F59F70F1F0F8019581907FD1F4DD
:103FB000D12C1EC090E0589FF001599FF00D1124A4
:103FC000E651FE4F6181361306C06081261303C09F
:103FD0006281E6120FC001968770D5CF9F7011F0F5
:103FE000882331F3805E883018F3C8010E947A1765
:103FF000FD2CB1CFEE2009F4AECF8091E8018160B5
:104000008093E801F12CA7CF431306C0921304C09C
:10401000F801EE2009F479C0C8010E94F40F88234A
:1040200009F1EE20F9F08091E801803270F02091E2
:10403000E3013091E40138872F831986DB86CA8635
:104040008C87CE0107960E947A1786E0F801A3EECE
:10405000B1E001900D928A95E1F70E94081FFF24BC
:10406000F39479CFC8010E947A17F9CF51110AC091
:1040700083EE91E00E947A1786E0F50111928A950D
:10408000E9F7C0CF43130FC092130DC0E1100BC06E
:10409000F8018583C8010E947A1786E0F501119224
:1040A0008A95E9F758CFC8010E94F40F8823D1F20E
:1040B000EE20C1F28091E801803238F22091E301D4
:1040C0003091E4013A8329831B82DD82CC828E8386
:1040D000CE010196B8CFE83CF105F8F6FE2CEE20B3
:1040E00009F243131FC092131DC08091E80180FDA7
:1040F00010C0982F907F69F0F8018583903F31F0D0
:10410000982F907F905F8F70892B8583C8010E94C4
:104110007A1786E0F801A3EEB1E001900D928A953E
:10412000E1F719CFC8010E94F40F81118ECF809161
:10413000E80181608093E801C8010E947A170BCFE3
:10414000EE2009F48FCFC8010E94F40FF82E8823C7
:1041500009F488CF86E0F801A3EEB1E001900D925A
:104160008A95E1F78091E3019091E4010E94E70FC5
:104170000E94081FF0CE81E08E25FBCEA7E1B0E0C3
:10418000E4ECF0E20C94EC294B8B5C8B6D8B7E8B1A
:104190008F8B611110923C021A8A198A85E0FE0108
:1041A0007396DE011D9601900D928A95E1F786E0E7
:1041B000FE013D96DE01179601900D928A95E1F77A
:1041C000CE0107960E945D1F882359F016E080916A
:1041D0001A029091E901891343C06796E3E00C94B9
:1041E000082A86E0FE013796DE01119601900D92B5
:1041F0008A95E1F78A859B85892B41F38F81988584
:1042000089238F3F19F32091E90130E0C90101961C
:104210008770992740911A024817190671F40E9475
:1042200090141092E90110921A0286E0E3EEF1E098
:10423000DF011D928A95E9F7C9CF96E0929FD001E0
:10424000939FB00D1124A651BE4FFE0131960190EF
:104250000D929A95E1F78093E9010E94550BB6CF34
:10426000819FC001112486519E4F0E945D1F8823AB
:1042700009F4B3CF80911A0290E0019687709927D4
:1042800080931A02A4CFA8E1B0E0E9E4F1E20C9433
:10429000E1298E010F5F1F4F88E1D8011D928A9599
:1042A000E9F72CE4E22E21E0F22ECC24C394D12CA9
:1042B00088248394912C51E6A52E51E0B52EF70168
:1042C00081917F018F3F09F449C0F894E82FE2956E
:1042D000EF70F0E021A18F70A40102C0440F551FC0
:1042E0008A95E2F7CA01922F982B91A392A180950B
:1042F000892382A3789400C095E5692E91E0792EF8
:10430000F801A60140955095D3016D913D01808142
:1043100091816F3F09F463C0262F22952F7030E002
:10432000D90190962C9130E06F7002C03595279599
:104330006A95E2F720FD53C08C299D2991838083E3
:104340003296A614B70401F7F701319780818F3FA9
:1043500011F00E940209B0EABA95F1F7CC0CDD1C0D
:10436000E5E5EE16E1E0FE0609F0A9CF48E150E0F0
:10437000B80183E492E00E94752A892B99F188E1C3
:10438000F801A3E4B2E001900D928A95E1F781E093
:10439000809342020E94180690934102809340024B
:1043A00080914002909141020E9409060597F0F029
:1043B00048E150E063E472E088E792E00E94752AE9
:1043C000892BC9F088E1E3E4F2E0A8E7B2E00190CC
:1043D0000D928A95E1F781E01092420208C0842391
:1043E0009523ACCF809142028111DACF80E06896AC
:1043F000EEE00C94FD2980E0EFCF90E080E00E9499
:104400002E2A883E9E4F19F40E941E10089580E0C7
:1044100008950E94FD2181110AC00E9425148091F7
:10442000E302847089628093E3020E94750F86E044
:1044300090E00E94202A8093E302803320F087706E
:1044400088628093E3029091E302892F817090FF4C
:1044500004C0892F8695869586950E945D060895ED
:104460001F920F920FB60F9211242F933F934F93E9
:104470005F936F937F938F939F93AF93BF93CF93EC
:10448000DF93EF93FF93D091E900DF708091EC0010
:10449000C82FC17080FDC0E81092E9008091F00043
:1044A000877F8093F00078940E94A6141092E90010
:1044B0008091F00088608093F000CD2BCF70C09386
:1044C000E900FF91EF91DF91CF91BF91AF919F9163
:1044D0008F917F916F915F914F913F912F910F90AD
:1044E0000FBE0F901F9018951F920F920FB60F924C
:1044F00011242F933F934F935F936F937F938F93E9
:104500009F93AF93BF93EF93FF938091E10082FF5E
:1045100009C08091E20082FF05C08091E1008B7F9D
:104520008093E1008091DA0080FF24C08091D80060
:1045300080FF20C08091DA008E7F8093DA00809126
:10454000D90080FF9DC080E189BD82E189BD09B4A9
:1045500000FEFDCF81E0809319038091F402811168
:1045600009C00E9481040E944C058091E200846091
:104570008093E2008091E10080FF17C08091E2000B
:1045800080FF13C08091E2008E7F8093E2008091D3
:10459000E20080618093E2008091D8008062809385
:1045A000D80019BC85E0809319038091E10084FF55
:1045B0002BC08091E20084FF27C080E189BD82E1A9
:1045C00089BD89B5982F917080FFFBCF8091D8006D
:1045D0008F7D8093D8008091E1008F7E8093E100F1
:1045E0008091E2008F7E8093E2008091E200816002
:1045F0008093E20080911A03882309F447C084E085
:1046000080931903809119038091E10083FF27C0F3
:104610008091E20083FF23C08091E100877F809337
:10462000E10082E08093190310921A038091E10067
:104630008E7F8093E1008091E2008E7F8093E20084
:104640008091E20080618093E20042E060E080E0DF
:104650000E941A058091F00088608093F000FF911D
:10466000EF91BF91AF919F918F917F916F915F91EA
:104670004F913F912F910F900FBE0F901F90189563
:1046800019BC109219031092F40274CF8091E300C8
:1046900087FD93E090931903B5CF78941F921FB6CE
:1046A0001F9211248F939F93AF93BF938091EB023E
:1046B0009091EC02A091ED02B091EE020196A11D45
:1046C000B11D8093EB029093EC02A093ED02B093A6
:1046D000EE02BF91AF919F918F911F901FBE1F90CF
:1046E00018951F921FB61F9211248F939F93AF931B
:1046F000BF938091EA02811113C08091EB029091E7
:10470000EC02A091ED02B091EE024196A11DB11D07
:104710008093EB029093EC02A093ED02B093EE0233
:10472000BF91AF919F918F911F901FBE1F901895C1
:10473000CDB7DEB7AA970FB6F894DEBF0FBECDBFD8
:1047400085B7806885BF85B7806885BF84B7877F58
:1047500084BF0FB6F894A89580916000886180931B
:104760006000109260000FBE80E890E00FB6F894F1
:1047700080936100909361000FBE80E099E0909378
:104780009701809396010E9481040E944C058091BC
:10479000E20084608093E20078948091190388237A
:1047A000A1F01091E9001F709091EC00892F8170A9
:1047B00090FD80E8182B1092E9008091E80083FDBD
:1047C0000E94A6141F701093E90082E084BD93E05C
:1047D00095BD9AEF97BD80936E000E941E108111C7
:1047E00002C00E94650F0CE411E075E5E72E71E050
:1047F000F72ED8018D918D018F3F11F00E94020993
:10480000E016F106B1F705E511E061E6E62E61E09C
:10481000F62EF80181918F018F3F11F00E9402095D
:10482000E016F106B1F788E1E8E7F2E0DF01282FB2
:104830001D922A95E9F7E3E4F2E0DF011D928A95E3
:10484000E9F70E94FD21811102C00E94251482E037
:1048500090E00E94202A80935E020E94371090937D
:10486000F0028093EF020E944321EFE3FCE93197CD
:10487000F1F700C000000E9443218091820280FF76
:1048800008C06FEF7FEF90E080E00E94522A0E9404
:10489000700C83E090E00E94202A0E9487123E9ACA
:1048A000469A3F9A479A259A2D9A269A2E9882E2FE
:1048B0008093800089E1809381008FEF9FEF909338
:1048C0008700809386000E9409220E94092280911D
:1048D0005B02811133C00E94FD21811104C00E943E
:1048E00025140E94A41188E090E00E94282A609379
:1048F000DE027093DF028093E0029093E1026E7F0C
:1049000071F40E94A41188E090E00E94282A60932C
:10491000DE027093DF028093E0029093E1020E9436
:104920001F071092A4028091DE0280FF04C060E0A5
:1049300086950E943D1181E080935B0280E091E0CA
:104940009093E7028093E60250E4252E442443949A
:104950008091190300E112E1853009F49FC00E94A3
:1049600043214FE5A42E42E0B42E08E712E0D8011F
:10497000F501219131918D919D9142E0E737F40746
:1049800009F49AC028173907A1F338E7832E32E0DB
:10499000932E512CD401ED90FD904D01F5016190C5
:1049A00071905F016E147F0459F16E247F24312CC5
:1049B000CC24C394D12CC3018C219D21892BB1F02F
:1049C0003EA25FA221E0C7018C219D21892B09F421
:1049D00020E028A70E9418068160782F9AA789A74F
:1049E0004EA15FA168A58AA50E94BE203394CC0C7D
:1049F000DD1CF9E03F12DFCFF5013297F182E08252
:104A000053942CE05212C6CF8FB7F8944091EB022A
:104A10005091EC026091ED027091EE028FBF6EC07A
:104A200080911903843049F180E00E945D0680E0A6
:104A30000E94CA0B1092EA0288E190E00FB6F89447
:104A4000A895809360000FBE2092600083B7817F9D
:104A5000846083BF83B7816083BF7894889583B770
:104A60008E7F83BF0FB6F894A8958091600088610F
:104A700080936000109260000FBE8091180388231D
:104A800069F00E944321E8E7F2E081919191892B3E
:104A900009F0C4C392E0E039F907B9F7809119032E
:104AA000853009F4BDCF0E9490140E9409220E9413
:104AB00050060E94CA0B53CF2817390709F065CF5B
:104AC0000E9418067C0180915C0290915D02E816BC
:104AD000F906A1F08FEF89A38AA31BA20E941806F2
:104AE0008160782F9DA38CA349A15AA16BA18DA1B0
:104AF0000E94BE20F0925D02E0925C028091A402CE
:104B00008823D1F18091A302E091DE02E695E81BB3
:104B1000E0939F02823009F03EC1F0E0EE57FD4F76
:104B2000E491EE2EF12C8AECC82E8EE0D82E8091E6
:104B3000A002882361F01092A0020E9418069093B0
:104B40009E0280939D021092A2021092A1020E94E6
:104B50001806E0919D02F0919E028E1B9F0B8F3FE5
:104B60009F4750F4EE0DFF1DF0939E02E0939D02CF
:104B70008DE992E0F601099586E0E7E9F2E0DE01D1
:104B8000119601900D928A95E1F710929902109278
:104B90009A0210929B0210929C028B819C81892B1D
:104BA00009F44AC080919502909196020E940906EC
:104BB0009C0190919102992309F454C32531310548
:104BC000D8F19F3F19F09F5F90939102FB80FF20E7
:104BD00059F00E9486089FEF1F140CF491E0899F02
:104BE000802D112480939902FC80FF2059F00E94AF
:104BF00086089FEF1F140CF491E0899F802D1124EB
:104C000080939A02309199023323B1F020919A0255
:104C1000222391F045EB3403C0011124992309F4B8
:104C200019C19093990245EB240390011124332379
:104C300009F413C130939A028D819E81892B09F466
:104C40004AC080919302909194020E9409069C01AF
:104C500090919002992309F400C321353105D8F1D0
:104C60009F3F19F09F5F90939002FD80FF2059F0C5
:104C70000E9464089FEF1F140CF491E0899F802D1F
:104C8000112480939B02FE80FF2059F00E9464084B
:104C90009FEF1F140CF491E0899F802D11248093C5
:104CA0009C0230919B023323B1F020919C0222237D
:104CB00091F045EB3403C0011124992309F4D0C0CD
:104CC00090939B0245EB240390011124332309F4B4
:104CD000CAC030939C0246E050E0BE016F5F7F4F38
:104CE00087E992E00E94752A892B61F480919902EC
:104CF00090919A02892B90919B02892B90919C0212
:104D0000892B11F00E94C40786E0FE013196A7E9C5
:104D1000B2E001900D928A95E1F70E9450069091C1
:104D20007702891779F0809377029FB7F8944091C2
:104D3000EB025091EC026091ED027091EE029FBF88
:104D40000E94CA0B80911903843009F001CE83E0E0
:104D50008093E9008091E80082FFFACD8091E8001D
:104D600090E085FF06C00E94A004882309F47EC05D
:104D700091E08091E8008B778093E800992309F413
:104D8000E7CDE981E150E33108F0F1C0F0E0E6560B
:104D9000F54D0C949F29863059F4F0E0E158FD4F11
:104DA000E491EE2EF12CBAEBCB2EBEE0DB2EBFCE83
:104DB000893061F4E695F0E0E458FD4FE491EE2E81
:104DC000F12CAEE2CA2EAEE0DA2EB1CE8F3061F415
:104DD000E695F0E0E758FD4FE491EE2EF12CF9EC6A
:104DE000CF2EFDE0DF2EA3CE853159F4F0E0EA5856
:104DF000FD4FE491EE2EF12CEBE7CE2EEDE0DE2E12
:104E000096CE38E2E32EF12C40E0C42E4DE0D42EB5
:104E1000883109F48CCE833249F4E4E7F2E0E5907E
:104E2000F49079E6C72E7EE0D72E81CE54EFE52EA2
:104E3000FF24F39469ECC62E6CE0D62E843209F47C
:104E400076CE90EDE92E97E0F92E2EE1C22E27E0E6
:104E5000D22E6DCE40929902E6CE40929A02ECCECE
:104E600040929B022FCF40929C0235CF80E2E82EE9
:104E7000F12CCE0101966C018091E80085FD0AC0FD
:104E80008091E8008B778093E8000E94A00488233B
:104E900099F36ECF8091F100D6018D936D01B1E051
:104EA000EB1AF10849F764CF1A828AE08B831AC0A3
:104EB0008A81823009F4C8C18330D9F1813009F088
:104EC00056C02FB7F8946091EB027091EC0280917C
:104ED000ED029091EE022FBF0E94A5296B837C8387
:104EE0008D839E8380911903843009F031CD109118
:104EF000E9001F709091EC00892F817090FD80E88F
:104F0000182B82E08093E9008091E80080FF0DC0BB
:104F100050E040E060E270E0CE0101960E94D104D2
:104F20008091E8008E778093E8001F701093E9006D
:104F30000FCDFE013196D8018C9111969C910E5F98
:104F40001F4F928383833296B2E000391B0799F793
:104F5000C9CF8A81823059F46B817C818D819E8199
:104F60000E94A52986E290E00E94342ABBCF8FEFF1
:104F70008983B8CF4C816B818A810E947B0F9827EF
:104F8000892798279E838D83ADCF2D813E8132273F
:104F9000232732274C816B818A810E94EE0EA2CF9B
:104FA0000E94140F9FCF8A81893061F48B81E5E0E4
:104FB0008E9FC00111246FEF70E00E945529862F4B
:104FC0000E9401078A81813809F1A8F4803809F02C
:104FD00089CF8B81FFEF8F9FC00111246FEF70E0AD
:104FE0000E945529462F20E06091E0028091DF0267
:104FF0000E94581077CF823859F1833809F072CF68
:1050000020E04091E1026C818B81F2CF60E08B81E6
:105010000E943D119B818091DE02911111C08E7F13
:105020008093DE021092A4022FEF40E782E021502D
:1050300040408040E1F700C000000E94940C52CF35
:1050400081608093DE0260E086950E943D114ACF28
:105050008B818093E20246CF8A81893089F08A3041
:10506000F1F0813851F1E8F4803809F03BCF8091BC
:10507000E102BFEF8B9FC00111246FEF70E00BC006
:105080008091E302869586958695AFEF8A9FC00151
:10509000112465E070E00E9455296B8323CF1B82A9
:1050A00021CF823891F0833809F01CCF8091DF0244
:1050B0008B838091E0028C8315CF8091DE0280FF8C
:1050C00002C08695F3CE80E0F1CE8091E202EECE72
:1050D0008091E3020E94750F6091DE027091DF0201
:1050E0008091E0029091E1020E944510FBCE80E1A8
:1050F0008A83F8CE1A8289E7D9CE0A811B811027CC
:1051000001271027FE0131967F01CC80CF018C0D45
:10511000911D6C01C80189579C4FEC14FD0409F4E2
:10512000E1CE0937110558F40E94202AD7011496C0
:105130008C930F5F1F4FFFEFEF1AFF0AEBCFF701C2
:105140001482F7CF0A811B81102701271027CE0177
:1051500001966C01EC80E00EF12EF11CC80189571C
:105160009C4F0E151F0509F4BDCE0937110528F413
:10517000D60114966C910E94342ABFEFCB1ADB0A39
:105180000F5F1F4FEBCF0E94DE0EACCE84E0B0CF9E
:105190000A811B81102701271027FE0131967F010C
:1051A000CC80CF018C0D911D6C01C8018796CE1467
:1051B000DF0409F497CE0036A3E01A0750F40E94EA
:1051C000202AF70184830F5F1F4FBFEFEB1AFB0A02
:1051D000ECCFD70114961C92F6CF0A811B811027C1
:1051E00001271027FE0131966F01EC80E00EF12EB1
:1051F000F11CC8018796E016F10609F473CE00365B
:10520000F3E01F0728F4D60114966C910E94342A0B
:10521000BFEFCB1ADB0A0F5F1F4FEBCF09BD19BDE4
:1052200009B400FEFDCF8091D8008F7D8093D80017
:105230008091E00082608093E0008091E00081FD39
:10524000FCCF0E9490142ACC86E290E00E94202A93
:105250001B821C821D828E8345CE2B30310508F0C7
:1052600001CD39CD2B30310508F0ADCCE5CCDB01DB
:105270008F939F930E94CA29BF91AF91A29F800DE7
:10528000911DA39F900DB29F900D1124089587FB4F
:10529000082E062687FD819567FD61950E94142AD8
:1052A0000EF4919507FC81950895AA1BBB1B51E153
:1052B00007C0AA1FBB1FA617B70710F0A61BB70B86
:1052C000881F991F5A95A9F780959095BC01CD012B
:1052D000089597FB072E16F4009407D077FD09D0A8
:1052E0000E94552907FC05D03EF4909581959F4F6B
:1052F0000895709561957F4F0895A1E21A2EAA1B1B
:10530000BB1BFD010DC0AA1FBB1FEE1FFF1FA21775
:10531000B307E407F50720F0A21BB30BE40BF50B72
:10532000661F771F881F991F1A9469F760957095FB
:10533000809590959B01AC01BD01CF010895EE0FC2
:10534000FF1F0590F491E02D09946927962769279E
:1053500078278727782708950E94B429332312F4E9
:105360008A1B9B0B0C94C529A29FB001B39FC0015F
:10537000A39F700D811D1124911DB29F700D811D81
:105380001124911D08950E94B429B7FF0895821B2E
:10539000930B08950E94B429A59F900DB49F900D82
:1053A000A49F800D911D11240895B7FF0C94CA2964
:1053B0000E94CA29821B930B08952F923F924F920D
:1053C0005F926F927F928F929F92AF92BF92CF9295
:1053D000DF92EF92FF920F931F93CF93DF93CDB79E
:1053E000DEB7CA1BDB0B0FB6F894DEBF0FBECDBF16
:1053F00009942A88398848885F846E847D848C84E7
:105400009B84AA84B984C884DF80EE80FD800C81EF
:105410001B81AA81B981CE0FD11D0FB6F894DEBFD2
:105420000FBECDBFED010895991B79E004C0991F0F
:10543000961708F0961B881F7A95C9F780950895EE
:10544000F999FECF92BD81BDF89A992780B508954C
:10545000A6E1B0E044E050E00C945A2AA8E1B0E0A4
:1054600042E050E00C945A2A262FF999FECF92BDC3
:1054700081BDF89A019700B4021639F01FBA20BD19
:105480000FB6F894FA9AF99A0FBE08950396272F4B
:105490000E94352A0E94342A252F0E94352A242F63
:1054A0000C94352A0196272F0E94352A0C94342A11
:1054B000DC01CB01FC01F999FECF06C0F2BDE1BDD4
:1054C000F89A319600B40D9241505040B8F70895C3
:1054D000FC014150504030F001900616D1F7319751
:1054E000CF010895882799270895FB01DC0104C0A6
:1054F0008D910190801921F441505040C8F7881BCC
:10550000990B0895F894FFCF8715AF155217AF1573
:105510005217E2150316521701170E17401B401BB6
:105520007B1B7B1B141C2E1CAA1BAA1B391CA61C34
:10553000B71CB71C54275827A927BA27C527D02737
:10554000D3272C286828B727B72777287A287D28DB
:0A555000A228C328C628C828ED28A9
:10555A000606300C0F0C0A0C050C050601191A1B5D
:10556A001C1D1E1F20212201020101818283E200EB
:10557A00E900EA00B500B600B700CD008301CC000F
:10558A008A019201940121022302240225022602A1
:10559A0027022A02B300B4006F0070009091929320
:1055AA0095949697343733323130C6F0F1F4F5F6E4
:1055BA00F700010202020206060609090909090999
:1055CA000F0F0F0F0F0F151515181919191919198A
:1055DA001919191923244022B684016201AC00FD6D
:0655EA0007160836080058
:00000001FF
